:04FFF00023001E00CC
:08FFF800000000000000000001
:03000000022FC804
:0C2FC80078FFE4F6D8FD75817E02300F22
:1036B60057502053657175656E63657200302E38FC
:0D36C600004A756E20323820323030360058
:0233EE008F2628
:1033F000E4F527F528C3E5289526E5279400502312
:10340000900000AF82AE83E4FCFD7B107A27F9F8D0
:10341000D31213304003A380EA0528E52870D605AF
:033420002780D230
:013423002286
:103508007BFF7A3679B61237421237D57F76123773
:10351800F57BFF7A3679C31237421237D57BFF7AAB
:093528003679C71237420237D58B
:102D480012377A1237B8123704E4F524E4F5257DF2
:102D580001AF251235587F011233EEE4FDAF25127D
:102D680035580525E525C3940340E40524E524C327
:102D7800940540D81237F27B017A01799C753600A8
:102D880075370CE4FFFE12336A90019CE064AB7067
:102D980004A3E064CD60391237E390019C74ABF072
:102DA800A374CDF0A37401F0E4A3F0A3F0A312136D
:102DB800BD3D4CCCCDE49001A5F0A304F0E4A3F014
:102DC8007B017A01799CF53675370CFFFE1233AC1E
:102DD80090019EE0D39405400374C0F0C39001A015
:102DE800E0943C90019FE094004006E4F0A3743B1B
:102DF800F020970B7D017F011230D4D2AF80FE9076
:102E0800019EE0FDE4FF1230D4D2AF123508E4F59C
:102E18000E123633D20EA296920BA297920C123350
:102E280026E50E60FCE4F50E12147912371A80F1CB
:0337F200C21622DA
:1035C800AD07AC062016FDD216EC5401F5F1EDF569
:1035D800F330AF0320EF0AE5F130E7FBC216AFF294
:0435E800227F00221C
:0434B200AB07AA06B4
:1034B6002016FDD216EA5401F5F1A2AF9200C2AF72
:1034C6008DF2EBF5F3A20092AF30AF0320EF07E5E4
:0634D600F130E7FBC21615
:0134DC0022CD
:04345800AB07AA060E
:10345C002016FDD216EA54014420F5F1A2AF9215C4
:10346C00C2AF8DF2EBF5F3A21592AF30AF0320EFA4
:08347C0007E5F130E7FBC21681
:013484002225
:10357E002016FDD21675F131A2AF9200C2AF8FF2B6
:10358E00E4F5F3A20092AF30AF0320EF07E5F13080
:04359E00E7FBC2166F
:0135A2002206
:0537DE00E4FD02345877
:0537E300E4FF02357E49
:0300730002000385
:0600030053F17FC216322A
:0A336A008E318F328B338A3489359F
:10337400E4F538F539C3E5399537E53895365027FE
:10338400E5322539FFE5313538FE1235C8AB33AAAD
:1033940034A935853982853883EF1211C40539E59E
:0733A4003970D2053880CE1C
:0133AB0022FF
:0A33AC008E318F328B338A3489355D
:1033B600E4F538F539C3E5399537E53895365027BC
:1033C600E5322539FFE5313538FEAB33AA34A93568
:1033D600853982853883121185FD1234B20539E5A7
:0733E6003970D2053880CEDA
:0133ED0022BD
:1031C700256C660025303264253032642E25303474
:1031D700642C25630025303364253032642E253076
:1031E70034642C256300252E33660025332E316683
:1031F70000244750524D422C412C302E30302C4C5D
:103207002C253033642C253033642C002C002C30D3
:1032170030302E302C00573A002C523A002C423ACC
:0132270000A6
:0437E8004101270074
:0A361000E0FF7E007B017A0079AB39
:10361A00EF7803C333CE33CED8F92420FFE43EFE3D
:09362A0075360075370802336A99
:1036D300EF7803C333CE33CED8F92420FFE43EFE84
:0936E3007536007537080233AC9E
:103228002094028028900126E004F0E0FF90019F9E
:10323800E0FCA3E0FDD39FEC940050359001A6E09C
:10324800601E24FE60248000900126EDF078AB7C9F
:10325800007D017B017A0179287E007F08021146F2
:1032680090019FA3E0900126F022E4900126F080CF
:0832780003900126123610221A
:10305400E4F531F532E53225E02457F8E4F608F6D4
:103064000532E532700205316414453170E7E4F548
:1030740031F53212116CFF600CB42009740129F986
:10308400E43AFA80EEEF6043AE02AF010532E53276
:10309400700205311425E02457F8A60608A6071285
:1030A400116CFF600D642C6009740129F9E43AFA8B
:1030B40080EDEF600CE41211B20429F9E43AFA80CD
:0F30C400028008E5326414453170A8AE31AF3296
:0130D30022DA
:10259D00753AFF753B31753CC7753D01753E01754B
:1025AD003F481222CCE4FBFA79C87842900148E00A
:1025BD00FCA3E0FDA3E0FEA3E0FF120CAD120E069E
:1025CD00900150EEF0A3EFF0900148E0FCA3E0FD88
:1025DD00A3E0FEA3E0FFC004C005C006C007900144
:1025ED0050E0FCA3E0FDE4120DCDE4FBFA79C878D0
:1025FD0042120BA4A804A905AA06AB07D007D00662
:10260D00D005D004120AAF9001481213B1900148C1
:10261D00E0FCA3E0FDA3E0FEA3E0FF120E06900197
:10262D0052EEF0A3EFF0900148E0FCA3E0FDA3E033
:10263D00FEA3E0FFC004C005C006C007900152E034
:10264D00FCA3E0FDE4120DCDA804A905AA06AB0775
:10265D00D007D006D005D004120AAF90014812134E
:10266D00B1900148E0FCA3E0FDA3E0FEA3E0FFE490
:10267D00FBFA79707842120BA49001481213B190B5
:10268D000152E0FCA3E0FDE4120DCDE4FBFA7970FC
:10269D007842120CADC004C005C006C007900150B1
:1026AD00E0FCA3E0FDE4120DCDD003D002D001D0AB
:1026BD0000120AB3C004C005C006C007E4FBFA79D6
:1026CD00617845900148E0FCA3E0FDA3E0FEA3E0A6
:1026DD00FF120CADD003D002D001D000120AB3907E
:1026ED00014C1213B1AB34AA35A93612116CFF642B
:1026FD00576004EFB4531790014CE0FCA3E0FDA329
:10270D00E0FEA3E0FF120DB790014C1213B1900142
:0C271D004CE0FCA3E0FDA3E0FEA3E0FF05
:01272900228D
:1035EC00753AFF753B31753CC7753D01753E0175EC
:1035FC003F371222CC900137E0FCA3E0FDA3E0FEA4
:03360C00A3E0FF39
:01360F002298
:082B08008F348E338D328C31C5
:102B10001237AB120E06900148EEF0A3EFF0AF347F
:102B2000AE33AD32AC311237ABC004C005C006C005
:102B300007900148E0FCA3E0FDE4120DCDA804A934
:102B400005AA06AB07D007D006D005D004120AAFFD
:102B5000E4FBFA79707842120BA490014E1213B183
:102B600090014EE0FCA3E0FDA3E0FEA3E0FF120E07
:102B70000690014AEEF0A3EFF090014EE0FCA3E0D6
:102B8000FDA3E0FEA3E0FFC004C005C006C007909F
:102B9000014AE0FCA3E0FDE4120DCDA804A905AABA
:102BA00006AB07D007D006D005D004120AAF9001BB
:102BB0004E1213B17F007E407D1C7C4690014EE09A
:102BC000F8A3E0F9A3E0FAA3E0FB120BA4120E06AF
:102BD00090014CEEF0A3EFF07538FF753931753A7E
:102BE000CB900148E0FEA3E08E3BF53CA3E0FEA3C2
:102BF000E08E3DF53EA3E0FEA3E08E3FF540E4FF0E
:102C0000FEFDFCAB34AA33A932A831120D4A5004A0
:102C10007F5380027F4E8F417B017A0079BC121A6C
:072C2000757B017A0079BC0D
:012C2700228A
:082C28008F348E338D328C31A4
:102C30001237AB120E06900148EEF0A3EFF0AF345E
:102C4000AE33AD32AC311237ABC004C005C006C0E4
:102C500007900148E0FCA3E0FDE4120DCDA804A913
:102C600005AA06AB07D007D006D005D004120AAFDC
:102C7000E4FBFA79707842120BA490014E1213B162
:102C800090014EE0FCA3E0FDA3E0FEA3E0FF120EE6
:102C90000690014AEEF0A3EFF090014EE0FCA3E0B5
:102CA000FDA3E0FEA3E0FFC004C005C006C007907E
:102CB000014AE0FCA3E0FDE4120DCDA804A905AA99
:102CC00006AB07D007D006D005D004120AAF90019A
:102CD0004E1213B17F007E407D1C7C4690014EE079
:102CE000F8A3E0F9A3E0FAA3E0FB120BA4120E068E
:102CF00090014CEEF0A3EFF07538FF753931753A5D
:102D0000DC900148E0FEA3E08E3BF53CA3E0FEA38F
:102D1000E08E3DF53EA3E0FEA3E08E3FF540E4FFEC
:102D2000FEFDFCAB34AA33A932A831120D4A50047F
:102D30007F5780027F458F417B017A0079BC121A50
:072D4000757B017A0079BCEC
:012D47002269
:1034DD007538FF753931753AEDE4FBFA797A784430
:1034ED00120CAD8F3E8E3D8D3C8C3B7B017A00796D
:0B34FD00BC121A757B017A0079BC221A
:103656007538FF753931753AF28F3E8E3D8D3C8C4B
:103666003B7B017A0079BC121A757B017A0079BC22
:013676002231
:10332600C210E49000B7F0900126F0123610E4FFC8
:10333600FE7D207C419001A1E0F8A3E0F9A3E0FA2C
:10334600A3E0FB120BA49000B81213B1E490011C89
:10335600F0C211A294B3920FA297B3920C900125DA
:04336600F00200264B
:10147900A20C309701B3500AA297920C209703123D
:101489003228900125E0600814F0E07003FD804ED9
:1014990012379CEF7003021A181236988F269001A2
:1014A900A7E06003200E05AF261237F5E52624F8DC
:1014B900603324FE604C24E6600C240360030219A7
:1014C900DFC20E0219D7E4900127F0E0FF04F0749F
:1014D900CC2FF582E43400F583E526F07D017F0207
:1014E90012355880AB900127E0D394004003E014F3
:1014F900F07F081235317F201235317F08123531DE
:10150900808E900127E024CCF582E43400F583E451
:10151900F0200E0ED20E7B017A0079CC121E8802C1
:1015290019D77B017A0079CE900134EBF0A3EAF068
:10153900A3E9F01213579001301213B17F437E4D86
:101549007D527C50900130E0F8A3E0F9A3E0FAA3C2
:10155900E0FBC312134660030219D77B017A0079B5
:10156900CC123054855C82855B83E0644160030260
:1015790019CAAA5DA95EC0038B34855F35856036BB
:10158900D00312259D9000A31213B1AA61A9627B11
:1015990001C0038B34856335856436D00312259DDC
:1015A9009000A71213B1AA67A9687B011235EC90C4
:1015B90001211213B12010499000B7E004F0E0C3F3
:1015C900940A50030219D7D2109000A3E0FCA3E0BB
:1015D900FDA3E0FEA3E0FF9001281213B19000A73C
:1015E900E0FCA3E0FDA3E0FEA3E0FF90012C1213B1
:1015F900B17D017F0212355890012574C8F0021996
:10160900D79000A7E0FCA3E0FDA3E0FEA3E0F53539
:101619008E348D338C32A3E0FCA3E0FDA3E0FEA35E
:10162900E0F5398E388D378C36A3E0FCA3E0FDA3B5
:10163900E0FEA3E0F53D8E3C8D3B8C3A753E01758D
:101649003F007540B375410175420175431D900016
:10165900A3E0FCA3E0FDA3E0FEA3E0FF1200769067
:101669000126E0FFD394004006EF14F52D80028F88
:101679002D7538FF753931753AF8753B00852D3C64
:10168900900126E0753D00F53E7B017A0079CC1288
:101699001A759000ABE0FCA3E0FDA3E0FEA3E0FF18
:1016A900122B088B318A3289337B017A0079CC126B
:1016B90032807531FF7532327533137B017A0079C7
:1016C900CC1232809000AFE0FCA3E0FDA3E0FEA3C2
:1016D900E0FF122C288B318A3289337B017A007919
:1016E900CC1232807531FF7532327533137B017A32
:1016F9000079CC1232809000B3E0FCA3E0FDA3E0B6
:10170900FEA3E0FF1234DD8B318A3289337B017A03
:101719000079CC1232807531FF7532327533137B03
:10172900017A0079CC12328090011DE0FCA3E0FD22
:10173900A3E0FEA3E0FF1236568B318A3289337B50
:10174900017A0079CC1232807531FF7532327533E6
:10175900157B017A0079CC123280A20F309401B343
:101769005006209403123228A294920F752756E44A
:10177900F5289001A5E07044E4FFFE7D7A7C449051
:1017890001A1E0F8A3E0F9A3E0FAA3E0FB120BA49E
:101799009000B3E0F8A3E0F9A3E0FAA3E0FB120D8F
:1017A9004A40030218777D017F02123558900125BE
:1017B9007464F07527411232280218772011030248
:1017C900184A9000B8E0FCA3E0FDA3E0FEA3E0FF07
:1017D9009000B3E0F8A3E0F9A3E0FAA3E0FB120D4F
:1017E9004A600A400890011CE004F08005E4900179
:1017F9001CF090011CE0D3940340307F031237683A
:10180900752741123228E4FFFE7D207C419001A119
:10181900E0F8A3E0F9A3E0FAA3E0FB120BA490001F
:10182900B81213B1C211E490011CF09000B3E0FCAE
:10183900A3E0FDA3E0FEA3E0FF9000B81213B1807E
:101849002DE4FFFE7D7A7C449001A1E0F8A3E0F944
:10185900A3E0FAA3E0FB120BA49000B3E0F8A3E025
:10186900F9A3E0FAA3E0FB120D4A5002D211753137
:10187900007532007533277B017A0079CC123280EA
:10188900E4F52CF52A752B017B017A0079CC12003D
:101899000EC3E52B9FEE6480F8E52A648098501901
:1018A90074CC252BF5827400352AF583E0622C056A
:1018B9002BE52B70D3052A80CF9001A7E070157B0B
:1018C900017A0079CC1237427F2A1237F5AF2C12F0
:1018D90036EC80647BFF7A32791D123742E52D049C
:1018E900FF1236EC7F2C1237F5900126E004FF1227
:1018F90036EC7BFF7A3279201237429000B3E0FC54
:10190900A3E0FDA3E0FEA3E0FF120E067B007A0030
:1019190079001228987BFF7A327924123742900194
:101929001DE0FCA3E0FDA3E0FEA3E0FF120E067B91
:10193900007A0079001228981237D5900121E0F831
:10194900A3E0F9A3E0FAA3E0FB90011DE0FCA3E00A
:10195900FDA3E0FEA3E0FF120AAF120E068E2A8F46
:101969002BD3E52B94B4E52A64809480400C7498B9
:10197900252BF52B74FE352AF52AC3E52B944CE566
:101989002A6480947F500C7468252BF52B740135DB
:101999002AF52AC3E52B9405E52A6480948050042E
:1019A9007D01801FD3E52B9405E52A64809480404E
:1019B90004E4FD80027D017F011235587D01E48038
:1019C90009E4FD7F01123558E4FDFF123558E49012
:1019D9000127F0021499900127E0FF04F074CC2F3D
:1019E900F582E43400F583E526F0900127E0B40A96
:1019F9000C900125E07006FD7F02123558900127F1
:0F1A0900E0C394505003021499E014F0021499B2
:011A180022AB
:10377A00E4F5847585FF53912FF592F5A475A5FF9D
:01378A00221C
:10370400C214E4FDFF123558E4FD7F01123558E47C
:06371400FD7F02023558A2
:10355800EF1460101460162402701ABD0103C2A78C
:1035680022D2A722BD0103C2A622D2A622BD0103F0
:06357800D28022C2802275
:10376800EF24FD700CD214750DFA7D017F0212351D
:023778005822D5
:10371A00E50DD39400400CD50D09C214E4FD7F02D7
:04372A0012355822DA
:1034240025640020200053657474696E67733A0044
:1034340041727269766552616E67653D00206D0068
:103444005365714D6F64653D004379636C654D6FE1
:0434540064653D006E
:061E88008B2E8A2F893029
:101E8E001235A3AB2EAA2FA93012116C900137F088
:101E9E0012141720C8411ED642205F43217C441ED7
:101EAE00D3451FA04C20774E2244502114511ECFF3
:101EBE005221AA532179561F0A57213F5900002259
:101ECE004D43A208220237E3AB2EE5302402F9E49B
:101EDE00352FFA753AFF753B34753C24753D017507
:101EEE003E01753F461222CC900146A3E090019E22
:101EFE00F0D39405400374C0F00220B8AB2EE53049
:101F0E002402F9E4352FFA123054AA57A9587B014E
:101F1E00C003753AFF753B34753C248B3D753E010D
:101F2E00753F46D0031222CCAA59A95A7B01C00391
:101F3E008B34855B35855C36D00312259D90013C34
:101F4E001213B1AA5DA95E7B01C0038B34855F3588
:101F5E00856036D00312259D9001401213B1900179
:101F6E0046E0FEA3E0FFD39400EE6480948050031D
:101F7E0002224DD3EF943CEE648094804003022203
:101F8E004DEF24FFFFEE34FFFE7B017A01793C0218
:101F9E0036D3E4900144F0A3F090019FE0FEA3E05D
:101FAE00FF900144E0FCA3E0FDC39FEC9E400302C2
:101FBE00224DC3ED943CEC64809480400302224D8C
:101FCE00900144E0FEA3E0FF7B017A01793C1236DA
:101FDE001A900145E02401FF900144E03400FE33E5
:101FEE0095E0FDFC7B007A0079001228987BFF7A41
:101FFE0034792712374290013CE0FCA3E0FDA3E0C8
:10200E00FEA3E0FF122B08900139EBF0A3EAF0A338
:10201E00E9F01237427BFF7A34792712374290016A
:10202E0040E0FCA3E0FDA3E0FEA3E0FF122C28900D
:10203E000139EBF0A3EAF0A3E9F01237421237D5DB
:10204E00900145E004F07006900144E004F0021F98
:10205E00A71237E3E490019FF0A3F07B017A017998
:10206E009CF53675370C0221A5AB2EE5302402F90E
:10207E00E4352FFA753AFF753B34753C24753D01F6
:10208E00753E01753F461222CC900146E0FEA3E05C
:10209E00FF90019FEEF0A3EFF0C3943CEE9400404E
:1020AE000990019FE4F0A3743BF07B017A01799CC7
:1020BE0075360075370CE40221A5AB2EE5302402EF
:1020CE00F9E4352FFA753AFF753B34753C24753DAE
:1020DE0001753E01753F461222CC900146E0FCA3ED
:1020EE00E0FDEC120DCDE4FBFA797A7844120CADDA
:1020FE009001A11213B17B017A01799C753600759E
:10210E00370CE40221A5AB2EAA2FA93090000212A3
:10211E001185B444089001A57401F08005E4900186
:10212E00A5F07B017A01799C75360075370CE48039
:10213E0066AB2EAA2FA93090000212118524CF6013
:10214E000E24DF601180009001A67401F0800DE472
:10215E009001A6F080069001A67402F07B017A0130
:10216E00799C75360075370CE4802C023508AB2E41
:10217E00AA2FA930900002121185B431089001A740
:10218E007401F08005E49001A7F07B017A01799C3F
:10219E0075360075370CE4FFFE0233AC7BFF7A34E4
:1021AE00792A1237421237D57BFF7A3479341237B7
:1021BE0042E4FFFE7D7A7C449001A1E0F8A3E0F9B1
:1021CE00A3E0FAA3E0FB120BA4120E067B007A002A
:1021DE0079001228987BFF7A3479411237421237F0
:1021EE00D57BFF7A3479441237429001A5E0700412
:1021FE007F4180027F441237F51237D57BFF7A3448
:10220E00794D1237429001A6E0600F24FE60130450
:10221E0070169001387448F0800E9001387431F0C9
:10222E0080069001387452F0900138E0FF1237F5B5
:0F223E001237D50237D57D017F011230D480FED3
:01224D00226E
:10002600E4F529F528F527F526AB29AA28A927A856
:1000360026AF29AE28AD27AC26120AAFC004C005EC
:10004600C006C007AB29AA28A927A826AF29AE282B
:10005600AD27AC26120AAFD003D002D001D00012D1
:0A0066000CAD8F0B8E0A8D098C087B
:01007000226D
:080076008F318E308D2F8C2E8E
:10007E009001371213BD3B5CA8F190013B1213BDEA
:10008E004AC2A72890013F1213BD29612E13900179
:10009E00431213BD42652EE0900137E0F8A3E0F95C
:1000AE00A3E0FAA3E0FBE4FFFE7D807C3F120AAFE3
:1000BE009001471213B1900143E0F8A3E0F9A3E0D9
:1000CE00FAA3E0FBAF31AE30AD2FAC2E120CAD1259
:1000DE0027BA900147E0F8A3E0F9A3E0FAA3E0FB0A
:1000EE00120BA490014B1213B1900143E0F8A3E060
:1000FE00F9A3E0FAA3E0FBAF39AE38AD37AC361258
:10010E000CAD1227BA900147E0F8A3E0F9A3E0FA8C
:10011E00A3E0FB120BA490014F1213B190014BE020
:10012E00FCA3E0FDA3E0FEA3E0FFA804A905AA0638
:10013E00FB120BA4E4FBFA7980783F120AB3122F5C
:10014E0022A804A905AA06AB07E4FFFE7D807C3F2A
:10015E00120CAD9001531213B190014BE0FCA3E0D1
:10016E00FDA3E0FEA3E0FF900153E0F8A3E0F9A3A6
:10017E00E0FAA3E0FB120BA49001571213B1900109
:10018E004FE0FCA3E0FDA3E0FEA3E0FFA804A90559
:10019E00AA06FB120BA4E4FBFA7980783F120AB38D
:1001AE00122F22A804A905AA06AB07E4FFFE7D8044
:1001BE007C3F120CAD90015B1213B190015BE0FC21
:1001CE00A3E0FDA3E0FEA3E0FF900153E0F8A3E05F
:1001DE00F9A3E0FAA3E0FB120BA490015F1213B196
:1001EE0090014FE0FCA3E0FDA3E0FEA3E0FF900131
:1001FE005FE0F8A3E0F9A3E0FAA3E0FB120BA490F2
:10020E0001631213B190014BE0FCA3E0FDA3E0FEED
:10021E00A3E0FF900163E0F8A3E0F9A3E0FAA3E006
:10022E00FB120BA49001671213B1AB35AA34A9339C
:10023E00A832AF3DAE3CAD3BAC3A120AAF90014393
:10024E00E0F8A3E0F9A3E0FAA3E0FB120CAD9001F5
:10025E006B1213B190019B740AF090016BE0FCA33A
:10026E00E0FDA3E0FEA3E0FF1227889001731213B6
:10027E00B190016BE0FCA3E0FDA3E0FEA3E0FF1252
:10028E0027729001771213B1900173E0FCA3E0FD89
:10029E00A3E0FEA3E0FF90015BE0F8A3E0F9A3E08A
:1002AE00FAA3E0FB120BA490014B1213B190015B69
:1002BE00E0FCA3E0FDA3E0FEA3E0FF900157E0F811
:1002CE00A3E0F9A3E0FAA3E0FB120BA4900177E000
:1002DE00F8A3E0F9A3E0FAA3E0FB120BA4A804A98B
:1002EE0005AA06AB07900163E0FCA3E0FDA3E0FEC8
:1002FE00A3E0FF120AAF90014F1213B190014FE02D
:10030E00FCA3E0FDA3E0FEA3E0FFA804A905AA0656
:10031E00FB120BA4C004C005C006C00790014BE041
:10032E00FCA3E0FDA3E0FEA3E0FFA804A905AA0636
:10033E00FB120BA4D003D002D001D000120AB312CC
:10034E002F2290017B1213B1900177E0FCA3E0FD08
:10035E00A3E0FEA3E0FF90015FE0F8A3E0F9A3E0C5
:10036E00FAA3E0FB120BA4900167E0F8A3E0F9A357
:10037E00E0FAA3E0FB120AB390017F1213B19001D1
:10038E007FE0FCA3E0FDA3E0FEA3E0F54B8E4A8DDB
:10039E00498C4890017BE0FCA3E0FDA3E0FEA3E0C6
:1003AE00FF1231549001931213B1900173E0FCA32C
:1003BE00E0FDA3E0FEA3E0FF90015FE0F8A3E0F90B
:1003CE00A3E0FAA3E0FB120BA490017BE0F8A3E0FC
:1003DE00F9A3E0FAA3E0FB120CAD9001971213B152
:1003EE00900197E0FCA3E0FDA3E0FEA3E0FF120D59
:1003FE00B7900197E0F8A3E0F9A3E0FAA3E0FB12AF
:10040E000BA4E4FBFA7980783F120AB390018712AD
:10041E0013B1900167E0FCA3E0FDA3E0FEA3E0FFB3
:10042E00A804A905AA06FB120AB39001831213B100
:10043E00E4FFFEFDFC900187E0F8A3E0F9A3E0FAEB
:10044E00A3E0FB120D4A603B4039900183E0FCA310
:10045E00E0FDA3E0FEA3E0FF120DB7900187E0F8E8
:10046E00A3E0F9A3E0FAA3E0FB120CAD90017FE04C
:10047E00F8A3E0F9A3E0FAA3E0FB120AB39001831C
:10048E001213B1900183E0FCA3E0FDA3E0FEA3E014
:10049E00FFA804A905AA06FB120BA4E4FBFAF9783F
:1004AE0040120BA4E4FBFA798078BF120AB39001D4
:1004BE008F1213B1E4FFFE7D407CC0900187E0F8FF
:1004CE00A3E0F9A3E0FAA3E0FB120BA4E4FBFA7994
:1004DE00807840120AB3900137E0F8A3E0F9A3E068
:1004EE00FAA3E0FB120BA4E4FBFA79807840120A1F
:1004FE00B3900187E0F8A3E0F9A3E0FAA3E0FB12C2
:10050E000BA4900137E0F8A3E0F9A3E0FAA3E0FB17
:10051E00120BA4E4FBFA79807841120CAD90018B9A
:10052E001213B190016BE0FCA3E0FDA3E0FEA3E08B
:10053E00FFA31213B190017FE0FCA3E0FDA3E0FE48
:10054E00A3E0FF90018FE0F8A3E0F9A3E0FAA3E0A7
:10055E00FB120BA490018BE0F8A3E0F9A3E0FAA341
:10056E00E0FB120BA4900183E0F8A3E0F9A3E0FAFC
:10057E00A3E0FB120AB390017BE0F8A3E0F9A3E03D
:10058E00FAA3E0FB120BA490018BE0F8A3E0F9A311
:10059E00E0FAA3E0FB120BA4900193E0F8A3E0F9BC
:1005AE00A3E0FAA3E0FB120AB3900197E0F8A3E0F0
:1005BE00F9A3E0FAA3E0FB120BA490016B1213B1A6
:1005CE0090018BE0F8A3E0F9A3E0FAA3E0FBE4FFCF
:1005DE00FE7D807C3F120AAF90016BE0F8A3E0F93C
:1005EE00A3E0FAA3E0FB120BA4900137E0F8A3E01E
:1005FE00F9A3E0FAA3E0FB120BA4C004C005C006E9
:10060E00C007AB35AA34A933A832AF3DAE3CAD3BE3
:10061E00AC3A120AAF900143E0F8A3E0F9A3E0FA76
:10062E00A3E0FB120CADD003D002D001D000120A11
:10063E00B390016B1213B190019BE014F090016B1B
:10064E00E0F8A3E0F9A3E0FAA3E0FBA3E0FCA3E04B
:10065E00FDA3E0FEA3E0FF120AAF1237AB90013FFD
:10066E00E0F8A3E0F9A3E0FAA3E0FB120D4A50096B
:10067E0090019BE0600302026890014FE0FCA3E052
:10068E00FDA3E0FEA3E0F54B8E4A8D498C48900108
:10069E004BE0FCA3E0FDA3E0FEA3E0FF123154907B
:1006AE0001671213B1900173E0FCA3E0FDA3E0FE1D
:1006BE00A3E0FF900153E0F8A3E0F9A3E0FAA3E072
:1006CE00FB120BA4C004C005C006C00790015BE07E
:1006DE00FCA3E0FDA3E0FEA3E0FF900157E0F8A32A
:1006EE00E0F9A3E0FAA3E0FB120BA4C004C005C01E
:1006FE0006C007900177E0FCA3E0FDA3E0FEA3E0B7
:10070E00FF900163E0F8A3E0F9A3E0FAA3E0FB1287
:10071E000BA4D003D002D001D000120AAF8F4B8EA3
:10072E004A8D498C48D007D006D005D004123154DA
:10073E007BDB7A0F79497840120AB390016312136A
:10074E00B1900147E0F8A3E0F9A3E0FAA3E0FBE4DF
:10075E00FFFE7D807C3F120CAD900147E0F8A3E0D8
:10076E00F9A3E0FAA3E0FB120CADE4FBFA79807872
:10077E00BF120AB3900187E0F8A3E0F9A3E0FAA351
:10078E00E0FB120BA4E4FBFA7980783F120AB31255
:10079E002F22E4FBFA7980783F120AB390016B1294
:1007AE0013B1E4FFFEFD7CC090016BE0F8A3E0F90D
:1007BE00A3E0FAA3E0FB120AB390016BE0F8A3E00A
:1007CE00F9A3E0FAA3E0FB120CAD90016B1213B18A
:1007DE0090016BE0F8A3E0F9A3E0FAA3E0FBE4FFDD
:1007EE00FE7D807C3F120AAF90018B1213B19001F7
:1007FE006BE0FCA3E0FDA3E0FEA3E0FF90016BE045
:10080E00F8A3E0F9A3E0FAA3E0FB120BA4E4FBFAD1
:10081E0079807840120CADE4FBFA7980783F120AA9
:10082E00B390018BE0F8A3E0F9A3E0FAA3E0FB128A
:10083E000CAD90018B1213B1E4FFFE7DC07C3E9097
:10084E00016BE0F8A3E0F9A3E0FAA3E0FB120BA41E
:10085E0090016BE0F8A3E0F9A3E0FAA3E0FB120B22
:10086E00A4E4FBFA798078BF120AB390016BE0F82A
:10087E00A3E0F9A3E0FAA3E0FB120BA490016F1220
:10088E0013B190017FE0FCA3E0FDA3E0FEA3E0FF27
:10089E0090018FE0F8A3E0F9A3E0FAA3E0FB120BBE
:1008AE00A490016B1213B190018FE0FCA3E0FDA3A5
:1008BE00E0FEA3E0FF90018FE0F8A3E0F9A3E0FAD9
:1008CE00A3E0FB120BA4A804A905AA06AB07E4FF3C
:1008DE00FE7D807C3F120AAF90015F1213B1900132
:1008EE007BE0FCA3E0FDA3E0FEA3E0FFA804A905C6
:1008FE00AA06FB120BA4E4FBFA79807840120BA433
:10090E00E4FBFA794078C0120AB390015FE0F8A3D5
:10091E00E0F9A3E0FAA3E0FB120BA4900183E0F848
:10092E00A3E0F9A3E0FAA3E0FB120BA490016FE0A1
:10093E00F8A3E0F9A3E0FAA3E0FB120BA4E4FBFAA0
:10094E0079C07840120CAD90016BE0F8A3E0F9A3EA
:10095E00E0FAA3E0FB120AAF90016FE0F8A3E0F912
:10096E00A3E0FAA3E0FB120BA4E4FBFA7980784033
:10097E00120CAD900183E0F8A3E0F9A3E0FAA3E036
:10098E00FB120AB390017BE0F8A3E0F9A3E0FAA30F
:10099E00E0FB120BA490016FE0F8A3E0F9A3E0FADC
:1009AE00A3E0FB120BA4900193E0F8A3E0F9A3E0FF
:1009BE00FAA3E0FB120AB390018BE0F8A3E0F9A3CF
:1009CE00E0FAA3E0FB120BA490013BE0F8A3E0F9E0
:1009DE00A3E0FAA3E0FB120BA4900147E0F8A3E01A
:1009EE00F9A3E0FAA3E0FB120BA490015F1213B17E
:1009FE0090015FE0FCA3E0FDA3E0FEA3E0FFAB3EB1
:100A0E00AA3FA940121377900143E0FCA3E0FDA397
:100A1E00E0FEA3E0FF900167E0F8A3E0F9A3E0FA9F
:100A2E00A3E0FB120BA4AB41AA42A943121377AB6E
:100A3E0041AA42A943121357E4FBFA79B478431240
:100A4E000D4A5022AB41AA42A943C003C002C001C5
:100A5E00121357E4FBFA79B47843120AAFD001D0DF
:100A6E0002D003121377AB41AA42A943121357E4E3
:100A7E00FBFAF9F8120D4A60244022AB41AA42A9B2
:100A8E0043C003C002C001121357E4FBFA79B478D5
:0D0A9E0043120AB3D001D002D00312137727
:010AAB002228
:0A37B800E4F5955396BF53A27F225B
:103633005389F0438901538FFE758C70E4F58A53E7
:10364300B8FD53B7FDD2A9D28C53890F4389905348
:033653008FEF22D4
:03000B000237CCED
:0937CC00050E758C70758A00323F
:10372E000D0A0030313233343536373839414243A1
:04373E0044454600B8
:1030D4005387BF75985053877FE4F5BABF01054302
:1030E400A240800353A2BFE4F5BDED146015146043
:1030F4001A14601F1460242404702575BEF075BF73
:103104000B802375BEF075BF05801B75BEF075BFBF
:1031140002801375BE7075BF01800B75BEB080034D
:1031240075BE30E4F5BF75BD035391FE4392014370
:1031340091025392FDC21753B8EF53B7EF43B8103F
:10314400E49000A1F09000A0F09000A2F0D2AC2294
:030023000232D8CE
:1032D800C0E0C083C082C0D075D010309830900054
:1032E800A1E0C3949F50259000A0E0FF04F0740073
:1032F8002FF582E43400F583E599F09000A1E0040D
:10330800F09000A0E0C394A04002E4F0C298309985
:0E33180004C299C217D0D0D082D083D0E03248
:103677007D207C4E7E0180027E00A217E4335E60CF
:103687000BED1D70011CED4C70EA80ECD2178F9981
:013697002210
:103485009000A1E0D394004021A3E0FF04F0740074
:103495002FF582E43400F583E0FF9000A1E014F0FD
:0C34A500A3E0C394A04005E4F0227F00E7
:0134B10022F8
:0337F50002367722
:103698007F207E4E9000A1E07010D3EF9400EE944E
:0D36A800004007EF1F70ED1E80EA12348510
:0136B50022F2
:1037420012116CFF600C1237F5740129F9E43AFA90
:0337520080EE22E4
:0F379C009000A1E0D3940040037F01227F002220
:1036EC00AB07EB54F0C4540F90373193FF1237F5FE
:0836FC00EB540F93FF0237F5B8
:0937D5007BFF7A37792E0237429E
:1035A30012116CFF601EC3648094E1400ED3EF647C
:1035B3008094FA5006EF24E01211B2740129F9E461
:0435C3003AFA80DC74
:0135C70022E1
:0E2898008F348E338D328C318B358A368937F2
:1028A600E4F542EC4D4E4F701EE94A4B70057F3001
:1028B6000237F5AB35AA36A937AF4205428F827586
:1028C600830074300229DCAE33AD32AC31EC3350C8
:1028D60036E5374536453570077F2D1237F58014B6
:1028E600AB35AA36A937AF4205428F82758300748D
:1028F6002D1211C4AF34AE33AD32AC311213228F68
:10290600348E338D328C31754101753B00753ACA70
:1029160075399A75383BE4FFFEFDFCAB3BAA3AA934
:1029260039A838D312134650030229C7AF34AE3341
:10293600AD32AC31A8381212908F3F8E3E8D3D8C51
:102946003CEC4D4E4F7004E541702CE53F2430F5CC
:1029560040E537453645357007AF401237F58014E8
:10296600AB35AA36A937AF4205428F82758300E59B
:10297600401211C4E4F541AF3BAE3AAD39AC38ABC9
:102986003FAA3EA93DA83C121205AA06A905A8041D
:10299600C3E5349FF534E5339AF533E53299F532DC
:1029A600E53198F531AF3BAE3AAD39AC38E47B0A48
:1029B600FAF9F81212908F3B8E3A8D398C3802292B
:1029C6001CE536453745356010AB35AA36A937853F
:0929D6004282758300E41211C471
:0129DF0022D5
:100AAC00020E72E86480F8E933E83360110460F0F8
:100ABC00ED33EC337009E8FCE9FDEAFEEBFF2204B0
:100ACC0060DED3EB9FEA9EE99DE8C2E78CF0C2F7AB
:100ADC0095F0400CE8CCF8E9CDF9EACEFAEBCFFB77
:100AEC00120E3D85D0F05804700320D5B3E8047085
:100AFC00075002B2D5020E7C92D5EC0460F7E4CC20
:100B0C00C0E0C398F8603B94186008400DD0E0FB3F
:100B1C00020E54E4FBFAC9FC8028E830E406E4C970
:100B2C00FBE4CAFCE830E305E4C9CACBFCE8540793
:100B3C006010F8C3E913F9EA13FAEB13FBEC13FC9E
:100B4C00D8F130F52FC3E49CFCEF9BFFEE9AFEED41
:100B5C0099FDD0E0FBEF4E4D4C701222DB03020EE0
:100B6C0079EC2CFCEF33FFEE33FEED33FDED30E78B
:100B7C00EB020E54EF2BFFEE3AFEED39FDD0E0FB0D
:100B8C0050130BBB0003020E7CED13FDEE13FEEFB6
:080B9C0013FFEC13FC020E54E0
:100BA400EC4D6011E8497017ED33EC3304600DE44B
:100BB400FCFFFEFD22E933E8330470F8020E7212E2
:100BC4000E3D58046009E4CC2481500628500902E3
:100BD4000E7C284003020E79C0E0EB4A7044B980D1
:100BE40006D0E0FB020E68EF4E701CBD8008EBFFE0
:100BF400EAFEE9FD80EBE98DF0A4FEE5F0020C8D40
:100C0400E9CDF9EAFEEBFFEF89F0A4FCE5F0CE892B
:100C1400F0A42EFFE435F0CD89F0A42DFEE435F0E8
:100C24008067EF4E7005BD80D780C3EF8BF0A4AC16
:100C3400F0EE8BF0A42CFCE435F0F8EF8AF0A42C51
:100C4400E5F038FCE433CB8DF0A42CFCE5F03BF864
:100C5400EE8AF0A42CFCE5F038F8E433CF89F0A454
:100C64002CFCE5F038CF3400CE89F0A42FFFE5F05A
:100C74003EFEE433C98DF0A42EFEE5F039CD8AF0B2
:100C8400A42FFFE5F03EFEE43DFD33D0E0FB50072A
:100C94000BBB000F020E7CEC2CFCEF33FFEE33FE9B
:060CA400ED33FD020E54C9
:100CAA00020E7CEC5D046005E859047003020E72C2
:100CBA00120E3D580460F6EC4860F2EC7004FDFE3A
:100CCA00FF22C860DB2481C85009C398600250061D
:100CDA00020E799850CAF582E9294B4A7005AB820F
:100CEA00020E6875F0007C1A7880C3EF9BEE9AEDCD
:100CFA0099400DC3EF9BFFEE9AFEED99FDE842F095
:100D0A00DC23ACF0D0E0FFD0E0FED0E0FDAB8220E7
:100D1A00E7101BEB60BAEC2CFCEF33FFEE33FEED71
:100D2A0033FD020E54E803F830E705C0F075F00011
:100D3A00EF2FFFEE33FEED33FD40B830E7C280AA55
:100D4A0074F8CC6480CCC86480C8F582046043C35C
:100D5A00EB9FF5F0EA9E42F0E99D42F0E89C45F0EF
:100D6A0060305018E5825FFFE582F42B5582FB5014
:100D7A00210ABA001D09B90019088016E5825BFB31
:100D8A00E582F42F5582FF50090EBE00050DBD0005
:100D9A00010CC3EB9FF5F0EA9E42F0E99D42F0E8B0
:0D0DAA009C45F06007CC4820E701B3EC2227
:100DB700ED33EC33600A047003BD8004ECB2E7FC4A
:010DC7002209
:100DC80075F020800E75F010800575F0087D007EA6
:100DD800007F003392D530D503121322EC33401034
:100DE800EF33FFEE33FEED33FDEC33FCD5F0ED22AF
:0E0DF800E5F0247EA2D513CC92E7CDCEFF22EB
:100E0600EDD2E7CD33EC3392D524814006E4FFFEE4
:100E1600FDFC22FCE4CFCECDCC24E0501174FF8043
:100E2600EDC3CC13CCCD13CDCE13CECF13CF0470E0
:070E3600F030D5DE021322AB
:101A1900E54C2438F8E6054C227835300702783849
:101A2900E475F0011213F702116C2000EB7F2ED23E
:101A3900008018EF540F2490D43440D4FF30040BA5
:101A4900EF24BFB41A0050032461FFE54D6002156D
:101A59004D0550E5507002054F30070D7835E47596
:101A6900F0011213F7EF0211B20235317403D207F4
:101A79008003E4C207F54C8B358A368937E4F54D86
:101A8900F54FF550E54D60077F20121A5480F57522
:101A99004EFFC201C200C202C203C205C206C20889
:101AA900121A22FF700D3007057F00121A65AF5018
:101AB900AE4F22B4255FC2D5C204121A22FF24D028
:101AC900B40A00501A75F00A784D30D50508B6FFEA
:101AD9000106C6A426F620D5047002D20380D924B3
:101AE900CFB41A00EF5004C2E5D204021D52D2014C
:101AF90080C6D20080C0D20280BCD2D580BAD205BD
:101B090080B47F20121A542002077401B54D004099
:101B1900F1121A19FF121A54021A8DD208D206802C
:101B290095121A19FB121A19FA121A19F94A4B7055
:101B39000679497A1E7BFF20022EE54D602A7E0038
:101B49008E8275830012118560060EEE654E70F067
:101B5900C2D5EBC0E0EAC0E0E9C0E0EE121DB2D0A8
:101B6900E0F9D0E0FAD0E0FB12116CFF60AAEBC0FB
:101B7900E0EAC0E0E9C0E0121A54D0E02401F9D04B
:101B8900E03400FAD0E0FBE54E0460DCD54ED980A4
:101B990087D20280A2121D9560F7E54E70010412EA
:101BA9000E87A94E600DE54E600914F54E121E3CD4
:101BB900EF60F3EA30E702F404C3995077EAF425B9
:101BC9004E0430E701E404F54E800D121D9560C105
:101BD900EA054E254E120E87EA784BF630E701E406
:101BE900254E04D54E0420050114121DB2E4C0E0AF
:101BF900121E3C784BE6601320E70714F6121A3CD4
:101C0900802204F6D0E014C0E07F00121A3CE54EB1
:101C19006007121A33154E800B300503121A33D0A0
:101C2900E0021A8DD0E00480C5121D9560A0E54E32
:101C390004120E87784BEAF6E54E2005026001048E
:051C49002404121DB28D
:101C4E0074FF04C0E0121E3C121A3CE54E20050241
:101C5E006003121A33D0E0B54EE87F45121A46786B
:101C6E004BE67F2B30E7047F2DF404C0E0121A54AC
:101C7E00D0E075F00A84C0F0121A3DD0E0121A3D81
:101C8E00021A8D791080027908C206C2088008D225
:101C9E00D5790A8004790AC2D5E54E047002F54E54
:101CAE00E4FAFDFEFF121A19FC7B08200113121A2A
:101CBE0019FD7B1030000A121A19FE121A19FF7B39
:101CCE0020EC3382D592D55013C3E43000069FFF2B
:101CDE00E49EFEE42001039DFDE49CFCE4CBF8C2EF
:101CEE0001EC700CCFCECDCCE824F8F870F3801751
:101CFE00C3EF33FFEE33FEED33FDEC33FCEB33FB82
:101D0E00994002FB0FD8E9EB300105F8D0E0C4484A
:101D1E00B201C0E00AEC4D4E4F78207B0070C2EA53
:101D2E00B54E0040BCC0E0121DB4D0F0D0E0200192
:101D3E0004C4C0E0C4B201C0F0121A3DD0F0D5F018
:101D4E00EB021A8D1214171B2A531C91581AFB4CB6
:101D5E001AF7421C954F1C9D441C9D491B10431C99
:101D6E00A3551BD4461C32451B9E471E69501AFFB5
:101D7E002D1B032E1B262B1B07231B24201E522A32
:101D8E001ABF4800001B1EE54EB4FF03754E061227
:101D9E001A19FC121A19FD121A19FE121A19FF78C5
:101DAE0044020EB6790AA2D5200314300509B910E3
:101DBE00020404B9080104A2D52006025001042031
:101DCE0002689202B54D005034C0E07F20300319F6
:101DDE007F30A20272067205500F121E0BC202C293
:101DEE0006C205C2087F30800F300503E9C0E0123D
:101DFE001A54300503D0E0F9D0E0B54DCC300517BC
:101E0E007F30B9100C121A547F583004077F788037
:101E1E0003B90803121A543002057F2D021A547F9B
:101E2E00202008F87F2B2006F322920280CF7F001D
:101E3E00B4070050052444F8E6FF22286E756C6C3A
:101E4E002900D201121A193001F8C201784D30D58D
:101E5E000108F6021ABF2D50434958121A192403CD
:101E6E00B405004001E4901E6493121A45743A12B0
:0A1E7E001A45D203754D04021C91B1
:10224E00E54C30030104F82328243AF8227837307D
:10225E000302783AE475F0011213F702116C60EC88
:10226E00C5507002154F14C550200304FF0237ED00
:10227E00783774FFF5F0021407FF023755E54D600D
:10228E0006D54D037F002220030F12378BEF600817
:10229E000550E5507002054F2278371213EE1211D9
:1022AE006CFF60E97837E475F0011213F780DE12E7
:1022BE002295EFC0E0122287D0E040F380A0D20337
:1022CE008002C2038B378A388939E4F54EF54CF516
:1022DE004FF550754D00C202C200C201C204122257
:1022EE005BFF7005AF4E7E0022B4253012225BFFDD
:1022FE0024D0B40A00500C75F00AC54DA4254DF536
:10230E004D80E924CFB41A00EF5002C2E5022569D0
:10231E00D20180D8D20080D4D20480D0EF1222878E
:10232E0050081222BDEF600E80A9EFC0E012229578
:10233E00D0E06F609EEF607412226C80A71222951F
:10234E00EF6069E54D7007054D8003122295EF6031
:10235E001420040E12224EE475F0011213F7EF1240
:10236E0011B2D54DE6200404054C054E80BA12225A
:10237E008BEFC0E0122287D0E0500412226CE4FFF3
:10238E0020040E12224EE475F0011213F7EF121113
:10239E00B2EF70DA200404054C054E808BE54D60DB
:1023AE0002054D1222BD12228BEF70C6300304E4DB
:1023BE0012226CE54E60030222F27EFF7FFF22E5C1
:1023CE004D6002054D1222BDD206D20512228BEFB0
:1023DE0030060260D7C0E012226CD0E0AC51AD5294
:1023EE00AE53AF54122E4B8C518D528E538F545080
:1023FE0007122295C20580D4200410200502054E36
:08240E0012224E1213EE054CE0
:102416001213770222E1D0E0809A7900800A7910BF
:10242600800679088002790AD205E54D6002054DDD
:10243600E9C0E01222BDEF60DD122295BF2D04D265
:10244600028003BF2B091222BDEF60CA12228BD075
:10245600E0B40A028033B40802802EBF302770022F
:102466007408C205C0E012228BD0E0BF7802800358
:10247600BF5816054DD54D028007D54D04D20580AF
:102486000B741080197002740ABF000AEFF8E4FC9E
:10249600FDFEFF02251CC0E0EF12226CD0E0F9E43D
:1024A600FCFDFEFFE9C0E0ECC0E0EDC0E0EEC0E000
:1024B600EFC0E012228BEFF8D0E0FFD0E0FED0E0D4
:1024C600FDD0E0FCD0F0E8604DB461004007B47B7D
:1024D600005002C2E524D0503DFA24F6500724F9F4
:1024E6005034240AFAEAB5F000502BCFA9F0A42FF5
:1024F600FF92D5E9C5F0CEA4A2D53EFE92D5E9C598
:10250600F0CDA4A2D53DFD92D5E9C5F0CCA4A2D5C7
:102516003CFCC205808EE8C0E020042A20050805A0
:102526004E30020312132212224E1213EE054C20D5
:10253600000B20010DEE8FF01211E68009121377C1
:102546008004EF1211B2D0E012226C0222E12004C4
:102556001012224E1213EE054CE54F8550F0121163
:10256600E680E812141723AB5324245823224C2365
:102576001E4222FA4824284F242C44234B4324206D
:1025860049242C5523CD4623CD4523CD4723262A42
:0725960025544E0000232A2A
:0D37AB00ED33EC3360065004EC6480FC222A
:102F1E00020E7222EDA2E7D2E7F9EC3340F260F333
:102F2E00B4FF08ED547F70E8020E7CF82481C2E0F5
:102F3E00C0E0F40428FAC313FCED92E7FD8C448D37
:102F4E00458E468F47EEA2E7E9BA7F02C3133400DF
:102F5E009400FA75F091A4E5F013F494FE8AF0A4AF
:102F6E0033E5F033248CD313FDE492E7FE7F007C2F
:102F7E003F758302ECC0E0F8EDC0E0F9EEC0E0FA78
:102F8E00EFC0E0FBAC44AD45AE46AF47120CADD042
:102F9E00E0FBD0E0FAD0E0F9D0E0F8120AB3ED642D
:102FAE0080FD30E7011CD583CBED33CC33F8D0E078
:0A2FBE00A2E71328C313CC13FD2271
:103154008F478E468D458C44AB4BAA4AA949A84853
:10316400120CAD122A008F478E468D458C44E548DB
:1031740030E747ECC0E0EDC0E0EEC0E0EFC0E0E4D3
:10318400FFFEFDFCAB47AA46A945A844120D4A7BA5
:10319400DB600250087A0F7949784080067A0F790B
:1031A4004978C0D0E0FFD0E0FED0E0FDD0E0FC12D2
:1031B4000AB38F478E468D458C44AF47AE46AD4526
:0331C400AC4422F6
:10272A003A70FA83BCAAE9E43E81E0F8BF9DE9E683
:10273A003F80000039283C1ABB9969663DA335E3FE
:10274A00BF255DE73FC90FDB418DDBCCC44936EEBF
:10275A0045C9913FC5B0F83D3F800000C317F53425
:10276A00452FFA73C60AFDDD12281904A2E1920068
:10277A001420E01590272A7404120FB98026122813
:10278A001930E102B20020E0EB8C448D458E468F71
:10279A004790273E7404120FB9A844A945AA46AB2C
:1027AA0047120BA4ED4C6007300004EC6480FC2255
:1027BA00122819C0E08C448D458E468F47902762B7
:1027CA007403120FB9A844A945AA46AB47120BA431
:1027DA00ECC544FCEDC545FDEEC546FEEFC547FF19
:1027EA009027527403120FB9D082A844A945AA4669
:1027FA00AB47E58230E007120CADB20080A6EFCB02
:10280A00FFEECAFEEDC9FDECC8FC120CAD8095EDD9
:10281A0033EC547FCC33920024605007D0E0D0E0F0
:10282A00020E727B837AF97922783E120BA4EDF9B3
:10283A0033ECF83324815011EFFBEEFA120E061234
:10284A000DC8ECB2E7FC120AB3ED33EC33602F2467
:10285A0003F8C313FCED92E7FDE82481E4501FEC72
:10286A00F8EDF9EEFAEFFB120E06EF04C2E0FCF502
:10287A0082120DD2ECB2E7FC120AB3E58203FAED3A
:0E288A0033EC3360071413FCED92E7FDEA22F5
:100E3D00E9D2E7C933E833F892D5EDD2E7CD33ECFB
:070E4D0033FC5002B2D52274
:100E5400EC30E7100FBF000C0EBE00080DBD0004FF
:100E64000BEB6014A2D5EB13FCED92E7FD2274FFAB
:100E7400FCFDFEFF22E480F8A2D574FF13FC7D8004
:030E8400E480EF18
:100E8700F920E72824F950037907E4F42402FB1832
:100E9700DBFDE624FB5014E9600DE4F618E604F6E2
:0F0EA700B40A08E4F6D9F57401F60A22C2D5227E
:100EB600ED33EC3392D5FA602AB4FF33EDC2E77B0B
:100EC600FF60067A0E79DBE4227A0E79E420D504F7
:100ED6007A0E79DF224E614E002B494E46002D498F
:100EE6004E4600E47A08F608DAFC7B00740722E82E
:100EF600C0E0ECC0E0EDC0E0EEC0E0EFC0E0EA75B7
:100F0600F010A4CAABF075F04DA42BFBE435F0FC51
:100F1600EA2410FAEB34C5FBEC34D9FCEDC2E7FF4A
:100F260075F056A4F42411C5F0F434C58FF0A42A44
:100F3600E5F03BE43CF620E714121036D0E0FFD093
:100F4600E0FED0E0FDD0E0FC120CAD8014F40412FB
:100F56001036D0E0FFD0E0FED0E0FDD0E0FC120B72
:100F6600A4D0E0F8E6FAEDD2E7CD33EC332482FBE9
:100F7600E4C3CF33CFCE33CECD33CD33DBF37B07D4
:100F860075F00A846004F6081B0AE5F0F6088FF08F
:100F9600740AA4FFACF08EF0740AA42CFEACF050D8
:100FA600010C8DF0740AA42CFDE435F0F608DBDEA6
:030FB6007407229B
:102E3800C207C208C209C20AF9E4F555F556FCFDF5
:102E4800FEFFE91006EA20090CB42D04D209D322AA
:102E5800B42B02D32224D0504794095041240A307D
:102E68000A15F88556F0740AA42872E74051C5F08F
:102E7800704D85F056D322D208C0E0E4FBFA7920E1
:102E88007841120BA4ECF8EDF9EEFAEFFBD0E0FC78
:102E9800E4120DD2120AB33007B41555D322240A0E
:102EA800200A20B4FE0720071AD207D32224EB6099
:102EB8000424E0700EA2099207D20AC209D322C3E1
:102EC800020E72E4300A0BE556300902F404A20738
:102ED80092093008EA255520D2E5A2E7920A500265
:102EE800F404B4260050D8CCC0E0EDC0E0EEC0E059
:102EF800EFC0E0EC121036D0E0FFD0E0FED0E0FDED
:102F0800D0E0FC200A05120BA48003120CAD300996
:062F180003120DB7C322F5
:100FB900C0E0EFFBEEFAEDF9ECF8120BA4D0E0F586
:100FC900F0EFFBEEFAEDF9ECF8121391A3A3A3A34A
:100FD900E8C0E0E9C0E0EAC0E0EBC0E0C0F0120B15
:100FE900A41213A1A3A3A3A3120AB3D0F0D0E0FBC8
:0D0FF900D0E0FAD0E0F9D0E0F8D5F0D42235
:1029E000BE1249253E4CCCCDBEAAAAAB3F8000000A
:1029F0003E7ADBB03EED63383F24BC7D3F490FDBC0
:102A0000ED33ECC2E7CC339200B4FF13ED547F609A
:102A100003020E727FDB7E0F7DC97C3F022AFBC260
:102A200001C3947F401E7007EDD2E794904015EFEC
:102A3000FBEEFAEDF9ECF87F007E007D807C3F1222
:102A40000CADD201ED33EC33248430E705E4C0E073
:102A5000806D04FAEDD2E754F0C333DAFD54073445
:102A6000002323C0E0CCC0E0F8EDC0E0F9EEC0E008
:102A7000FAEFC0E0FBE4120DD2EC24FEFC8C4C8D8E
:102A80004D8E4E8F4F120BA47B007A007980783FD9
:102A9000120AB3ECC54CB2E7FCEDC54DFDEEC54ED8
:102AA000FEEFC54FFFD0E0FBD0E0FAD0E0F9D0E078
:102AB000F8120AB3A84CA94DAA4EAB4F120CAD8C1C
:102AC0004C8D4D8E4E8F4F9029E07403120FB9A894
:102AD0004CA94DAA4EAB4F120BA4D0E0600F24ECD2
:102AE000F582E43429F5831213A1120AB330010BE5
:102AF0007BDB7A0F79C978BF120AB3ED33EC336010
:082B000006ECA20092E7FC22A2
:101006003F8000004120000042C80000447A0000F2
:10101600461C400047C35000497424004B18968074
:101026004CBEBC205A0E1BCA6753C21C749DC5AE6B
:10103600FB60065407601C2323121064EB543860CF
:101046000912105012105F120BA4ECF8EDF9EEFA2B
:10105600EFCB22EB12105F80F1543803241C901062
:1010660006FE93FC0EEE93FD0EEE930ECE93FF223C
:102FD400022D48E493A3F8E493A34003F68001F29E
:102FE40008DFF48029E493A3F85407240CC8C333FE
:102FF400C4540F4420C8834004F456800146F6DFCD
:10300400E4800B01020408102040809037E8E47E3D
:10301400019360BCA3FF543F30E509541FFEE493C1
:10302400A360010ECF54C025E060A840B8E493A388
:10303400FAE493A3F8E493A3C8C582C8CAC583CAB3
:10304400F0A3C8C582C8CAC583CADFE9DEE780BE6B
:0137EC0000DC
:10107600E709F608DFFA8046E709F208DFFA803E5C
:1010860088828C83E709F0A3DFFA8032E309F60849
:10109600DFFA8078E309F208DFFA807088828C83B1
:1010A600E309F0A3DFFA806489828A83E0A3F60865
:1010B600DFFA805889828A83E0A3F208DFFA804C3F
:1010C60080D280FA80C680D4806980F28033801016
:1010D60080A680EA809A80A880DA80E280CA80337F
:1010E60089828A83ECFAE493A3C8C582C8CCC583F7
:1010F600CCF0A3C8C582C8CCC583CCDFE9DEE780C7
:101106000D89828A83E493A3F608DFF9ECFAA9F045
:10111600EDFB2289828A83ECFAE0A3C8C582C8CC9B
:10112600C583CCF0A3C8C582C8CCC583CCDFEADEB4
:10113600E880DB89828A83E493A3F208DFF980CC16
:1011460088F0EF60010E4E60C388F0ED2402B4040F
:101156000050B9F582EB2402B4040050AF232345B6
:0611660082239010C67305
:10116C00BB010689828A83E0225002E722BBFE0281
:09117C00E32289828A83E49322B4
:10118500BB010CE58229F582E5833AF583E022501F
:1011950006E92582F8E622BBFE06E92582F8E22269
:0D11A500E58229F582E5833AF583E4932283
:1011B200BB010689828A83F0225002F722BBFE011C
:0211C200F32216
:1011C400F8BB010DE58229F582E5833AF583E8F061
:1011D400225006E92582C8F622BBFE05E92582C80D
:0211E400F222F5
:1011E600BB010A89828A83F0E5F0A3F0225006F754
:0F11F60009A7F01922BBFE06F3E5F009F3192251
:10120500E88FF0A4CC8BF0A42CFCE98EF0A42CFC88
:101215008AF0EDA42CFCEA8EF0A4CDA8F08BF0A406
:101225002DCC3825F0FDE98FF0A42CCD35F0FCEB65
:101235008EF0A4FEA9F0EB8FF0A4CFC5F02ECD392A
:0F124500FEE43CFCEAA42DCE35F0FDE43CFC2297
:1012540075F008758200EF2FFFEE33FECD33CDCC51
:1012640033CCC58233C5829BED9AEC99E5829840D4
:101274000CF582EE9BFEED9AFDEC99FC0FD5F0D6B1
:10128400E4CEFBE4CDFAE4CCF9A88222B800C1B9DB
:101294000059BA002DEC8BF084CFCECDFCE5F0CB19
:1012A400F97818EF2FFFEE33FEED33FDEC33FCEB52
:1012B40033FB10D703994004EB99FB0FD8E5E4F90D
:1012C400FA227818EF2FFFEE33FEED33FDEC33FCFA
:1012D400C933C910D7059BE99A4007EC9BFCE99AEE
:1012E400F90FD8E0E4C9FAE4CCFB2275F010EF2F33
:1012F400FFEE33FEED33FDCC33CCC833C810D70733
:101304009BEC9AE899400AED9BFDEC9AFCE899F86D
:0E1314000FD5F0DAE4CDFBE4CCFAE4C8F92200
:0E132200C3E49FFFE49EFEE49DFDE49CFC22DC
:10133000EB9FF5F0EA9E42F0E99D42F0EC6480C834
:0613400064809845F022D4
:10134600EB9FF5F0EA9E42F0E99D42F0E89C45F0FD
:011356002274
:10135700BB010789828A830214495005E9F8021400
:101367003DBBFE05E9F802145589828A8302139171
:10137700BB010789828A830213B15005E9F8021479
:0A13870061BBFE05E9F802146D22B7
:10139100E493FC740193FD740293FE740393FF22A2
:1013A100E493F8740193F9740293FA740393FB22A2
:0C13B100ECF0A3EDF0A3EEF0A3EFF022AF
:1013BD00A8828583F0D083D0821213D41213D41255
:1013CD0013D41213D4E473E493A3C583C5F0C5837A
:1013DD00C8C582C8F0A3C583C5F0C583C8C582C87A
:0113ED0022DD
:0913EE00E6FB08E6FA08E6F92224
:1013F700FAE6FB0808E6F925F0F618E6CA3AF622F7
:10140700FAE6FB0808E625F0F9F618E63AFAF622B6
:10141700D083D082F8E4937012740193700DA3A364
:1014270093F8740193F5828883E473740293686078
:06143700EFA3A3A380DF78
:10353100EFB40A07740D12353C740A309811A8993A
:10354100B8130CC2983098FDA899C298B811F630FA
:0735510099FDC299F59922D2
:10378B0010180B1237C2BF0D027F0A023531AF0F73
:01379B00220B
:0537ED008F0FD218222D
:10375500EFC394094005EF940E4003BF2003D380C7
:0337650001C3227B
:103280008B2E8A2F89308B348A358936AB2E0530C8
:10329000E530AA2F7002052F14F912116C70ED742D
:1032A000FF2530F53074FF352FF52FAB310533E5B1
:1032B00033AA327002053214F912116CFFAB2E05DD
:1032C00030E530AA2F7002052F14F9EF1211B270F9
:0832D000DAAB34AA35A936225D
:10000E00E4FFFE12116C600C0FEF70010E09E97027
:05001E00F20A80EF2250
:0C143D00E6FC08E6FD08E6FE08E6FF22DB
:0C144900E0FCA3E0FDA3E0FEA3E0FF2216
:0C145500E2FC08E2FD08E2FE08E2FF22D3
:0C146100ECF608EDF608EEF608EFF622B7
:0C146D00ECF208EDF208EEF208EFF222BB
:0A37C2003098FDAF99C2987E0022F6
:00000001FF
